:020000040000FA
:020000001828BE
:08000800A4008B138C1E0628D6
:100010008C121A08A10011202108870024088B17D0
:1000200009000310A10D031C08000130A100080005
:1000300003179E019F0103138B170B1783168C1652
:1000400083128C1283160030870000308600FF3048
:1000500085001930990018159816181283129817F0
:100060001816860187010130A1000714851936286A
:100070003C200710452035280C1E3C2821089900FB
:100080008316981C412883120800A20B4528A30B55
:0400900045280800F7
:02400E00D430AC
:00000001FF
